:020000002E2CA4
:08000800FF00030E8312031335
:10001000B4000A0EB500040EB6008A110A12562C5E
:100020000130E507E50CFF30E50500000000E50BB9
:1000300015280800E208031D1E280800F9300000FA
:1000400000000000000000000000FF3E031D1F280C
:100050000000000000000000000000000000E20BB3
:100060001E280800650893008316141C3428080015
:100070001830831603130504850018308312050514
:10008000DE0059085E0603190800C830E50010209C
:100090001830831605048500183083120505D20038
:1000A0005E085206031D08005908083A0319622821
:1000B000183A03197928083A03199028183A0319AD
:1000C000A828BF28D208031D6D28CB08CB0DCB0D67
:1000D000FC30CB055208CB04BF285208183A031D48
:1000E000BF28D108D10DD10DFC30D1055208D10463
:1000F000BF285208183A031D8528CB08CB0DCB0D1D
:10010000FC30CB055208CB04BF28D208031DBF2802
:10011000D108D10DD10DFC30D1055208D104BF2832
:100120005208083A031D9C28CB08CB0DCB0DFC30A0
:10013000CB055208CB04BF285208103A031DBF2834
:10014000D108D10DD10DFC30D1055208D104BF2802
:100150005208103A031DB428CB08CB0DCB0DFC3050
:10016000CB055208CB04BF285208083A031DBF280C
:10017000D108D10DD10DFC30D1055208D10452085F
:10018000D9000800831203130613061708007F30F6
:1001900083160313060586007F308312060586004A
:1001A0005008E50032207F30060586007F3083123C
:1001B0000605E5008030650486000130E50010206A
:1001C00008008312031349030319080038204B0861
:1001D000CC005108E0004B08583A031D0929550886
:1001E00050020318F82850085502C800C803FD281B
:1001F0005003E50055086502C8005008480203187E
:100200000529D0035508D0020629D001C801C7200E
:10021000CB015108383A031D08005008C800E50119
:10022000C80A0319E50A5508C80748085002031808
:100230002129D008E501D00A0319E50A5508D0079D
:100240002329FF30D000C801C720D1010800831244
:10025000031306130930E5003220FF308312E50056
:100260003220C220080083160313861406110612DA
:1002700086130613831286170617403083169400E0
:1002800083129401941608000430831603139F0010
:1002900005088312E4000230831605048500C93086
:1002A00083129F00E5012830650203185929E50AE9
:1002B000532904301F049F001F195C29640883160A
:1002C000850007309F0083129F0108000E308316BF
:1002D00003139F0005088312E40001308316050410
:1002E0008500C13083129F00E501283065020318A4
:1002F0007B29E50A752904301F049F001F197E29F8
:1003000064088316850007309F0083129F01080050
:10031000EB01EE01EF016608EC00ED01EB190800BE
:10032000671C98296C08EE070318EF0A6D08EF07A1
:10033000E70C0310EC0DED0DEB0A8E29EC01ED013D
:10034000EF01F001EE016E1A08000310EF0DF00D41
:10035000E20DE30DEC0DED0D65086D02031DB229F4
:1003600064086C02031CBB296408EC026508031CCA
:10037000ED03ED026F14EE0AA329E1205B0ADB0016
:100380005B08E500322083125B08013A0319DE297D
:10039000033A0319E229013A0319E929073A031933
:1003A000ED29013A0319F429033A0319F829013A0E
:1003B0000319FC290F3A0319002A032A4D08E50006
:1003C0003220032A80304E04CE004E08E500322051
:1003D000032A4F08E5003220032A80305404D40059
:1003E0005408E5003220032A5708E5003220032A8A
:1003F0005808E5003220032A5C08E5003220032A71
:100400005F08E5003220C2202721E40106305B02AC
:100410000319E40AE4080319BD29DB01080083126B
:100420000313E501E50ACA08031D6510E401E40AA7
:10043000DD08031D6410640865050319242A0130D2
:10044000DD00460AC6002C2A043083160504850008
:10045000043083120505CA0046080F3A031D622ABC
:10046000E70104304A020319E70AE6015D030319B4
:10047000E60A660867050319632ADD01C60147031A
:100480000319632A55080E3A031D522AD50101307B
:10049000C700DF30831606058600DF3083120605AD
:1004A0008600632A0E30D5000130C700DF30831686
:1004B00006058600DF3083120605E8002030680458
:1004C0008600632ADD01CA0108003321403083160B
:1004D00006058600831206170F30E50032208312CE
:1004E000E5013220C2200C30E500322001308312B9
:1004F000E5003220C2200B30E500322005308312A7
:10050000E5003220C2200930E50032203F3083125E
:10051000E5003220C2200A30E50032200F3083127D
:10052000E5003220C2200800831203133B08F73A8B
:10053000BC1F013003193C06031DB62AFD3083168B
:1005400006058600FD30831206058600D001C7200F
:10055000F730831606058600F73083120605E200A1
:100560000830620486000130DA000800DA01FD304C
:10057000831606058600FD3083120605E200023070
:1005800062048600F730831606058600F730831272
:1005900006058600080044211E08E200E301E20D82
:1005A000E30DE20DE30DFC30E20583161E0C831211
:1005B000E400E40CE40E03306405E204E30862089E
:1005C000E4006308E500080066211E08E200E3017C
:1005D000E20DE30DE20DE30DFC30E20583161E0C87
:1005E0008312E400E40CE40E03306405E204E30843
:1005F0006208E4006308E50008000730831603136F
:100600009F00C03081008312D001D501D901D101F2
:10061000652283168601831286013D308316060506
:1006200086003D3083120605E200C2306204860077
:10063000C701E4226408B9006508BA00B9083A089D
:10064000E2003A0DE20CB90C3A0DE20CB90C62086A
:10065000BA00E6013908E2003A08E300BA1F362B77
:10066000E209E309E20A0319E30AE60A6430E40056
:10067000E5019E216F08CD00661C402BCD09CD0AF7
:10068000EB013908E2003A08E300BA1F4D2BE209FA
:10069000E309E20A0319E30AEB0A0A30E400E50180
:1006A0009E216F08CE007008EA006B1C5C2BCE09FF
:1006B000EA09CE0A0319EA0A4D08E6000A30E70003
:1006C00088216E08E8006F08E9006808CE024E082D
:1006D000E6000A30E70088216E08E2006F08E300B8
:1006E00062083902CF00630A031863083A02E8007F
:1006F0004D08E6006430E70088216E08E4006F08CA
:10070000E5006408CF02CB226408BB006508BC008A
:10071000BB083C08E2003C0DE20CBB0C6208BC00CC
:10072000E6013B08E2003C08E300BC1F9D2BE20908
:10073000E309E20A0319E30AE60A6430E400E5018A
:100740009E216F08D400661CA72BD409D40AEB01A4
:100750003B08E2003C08E300BC1FB42BE209E309BC
:10076000E20A0319E30AEB0A0A30E400E5019E21DC
:100770006F08D7007008EA006B1CC32BD709EA0981
:10078000D70A0319EA0A5408E6000A30E70088216C
:100790006E08E8006F08E9006808D7025708E6000D
:1007A0000A30E70088216E08E2006F08E300620863
:1007B0003B02D800630A031863083C02E8005408AF
:1007C000E6006430E70088216E08E4006F08E50069
:1007D0006408D8029422DA08031D062CC901E3013B
:1007E0003908530203193A08031DE30AE2013B08E2
:1007F000560203193C08031DE20A62086305031947
:10080000032CBD21042CE1200F22182BE101103014
:1008100061020318182B0130C900BD210230E2002B
:100820001A20F730831606058600F7308312060576
:1008300086000130E2001A20BD21F730831606053C
:100840008600F73083120605E20008306204860055
:100850000230E2001A20C901E10A072CD5308312C8
:100860000313A000C430A100BB30A200DC30A30001
:10087000A401A501A601A701A801A901AA01AB0134
:10088000AC01AD01AE01AF01C001C101B701B801BA
:10089000C201C301C401C501B001B101B201B3017C
:1008A000BE01BF01BD018A110A12FD2A8312031382
:1008B000360E8400350E8A00340E8300FF0E7F0E44
:0208C00009002D
:02400E00AA3FC7
:00000001FF
